:05000000020033815AEB
:02000B00815B17
:0200130081BBAF
:02001B0081BCA6
:0200230081BD9D
:02002B0081BE94
:10003300759840758780758921758DFF758BFF7560
:100043008850D29975816075A8827530007531002A
:10005300D210D211D212D213D214D215D216D21771
:10006300D218D219D21AD21BD21CD21DD21ED21F21
:10007300D220D221D222D223D224D225D226D227D1
:10008300D228D229D22AD22BD22CD22DD22ED22F81
:10009300D230D231D234D235D236D237D240D24115
:1000A300D242D243D244D245D246D247D248D24991
:1000B300D24AD24BD24CD24DD24ED24FD250C25151
:1000C300D290209014301021C210B21120110512C9
:1000D30004CD80151204EF801020100DD2102011D2
:1000E300051204EB800312050DD2912091143012F6
:1000F30021C212B213201305120511801512052E09
:10010300801020120DD21220130512052A8003122B
:100113000547D292209214301421C214B21520152F
:100123000512054B8015120587801020140DD2147B
:1001330020150512056980031205A5D29320931497
:10014300301621C216B2172017051205C3801512E7
:1001530005FF801020160DD2162017051205E18029
:100163000312061DD294209414301821C218B21918
:1001730020190512063B8015120677801020180DF2
:10018300D2182019051206598003120695D295201C
:100193009514301A21C21AB21B201B051206B38014
:1001A300151206EF8010201A0DD21A201B05120615
:1001B300D1800312070DD296209614301C21C21C45
:1001C300B21D201D0512072B801512076780102012
:1001D3001C0DD21C201D051207498003120785D26E
:1001E30097209714301E21C21EB21F201F0512072D
:1001F300A380151207CF8010201E0DD21E201F05CD
:100203001207B980031207E5D2A020A014302021E1
:10021300C220B2212021051207FB80151208188085
:100223001020200DD220202105120814800312086B
:1002330031D2A120A114302221C222B223202305CE
:100243001208358015120852801020220DD2222068
:10025300230512084E800312086BD2A220A2143089
:100263002421C224B22520250512086F8015120807
:100273008C801020240DD2242025051208888003A9
:100283001208A5D2A320A314302621C226B2272008
:1002930027051208A980151208C6801020260DD242
:1002A300262027051208C280031208DFD2A420A447
:1002B30014302821C228B2292029051208E3801509
:1002C300120900801020280DD2282029051208FCCD
:1002D3008003120919D2A520A514302A21C22AB2FB
:1002E3002B202B0512091D801512093A8010202A94
:1002F3000DD22A202B051209368003120953D2A6E8
:1003030020A614302C21C22CB22D202D0512095702
:1003130080151209748010202C0DD22C202D05126B
:100323000970800312098DD2A720A714302E21C291
:100333002EB22F202F0512099180151209AE8010BD
:10034300202E0DD22E202F051209AA80031209C7D1
:10035300D2B020B014303021C230B2312031051276
:1003630009CB80151209DD801020300DD2302031E9
:10037300051209D980031209EBD2B220B21430342A
:1003830021C234B2352035051209EF8015120A0156
:10039300801020340DD2342035051209FD8003125C
:1003A3000A0FD2B320B314303621C236B237203706
:1003B30005120A138015120A25801020360DD23635
:1003C300203705120A218003120A33D2B420B41C49
:1003D300753207120A371204BFD53206753201127D
:1003E3000A371204C6D2B420B40280EDD2B520B5C8
:1003F3001C753207120A4F1204BFD532067532013B
:10040300120A4F1204C6D2B520B50280EDD2B6202F
:10041300B61C753207120A671204BFD5320675324D
:1004230001120A671204C6D2B620B60280EDD2B713
:1004330020B71C753207120A821204BFD532067523
:100443003201120A821204C6D2B720B70280ED43EA
:10045300870101C302003332C0D0C0E0C083C08231
:10046300305010C250C281D251753300753400D25E
:10047300808018205115B2800533E533900A9D938F
:10048300F58CD082D083D0E0D0D032B2800534E571
:1004930034B4FF10C251D280758CFFD082D083D088
:1004A300E0D0D032B40A02D281900B9D93F58CD068
:1004B30082D083D0E0D0D032323232327E20DFFE9F
:1004C300DEFC227E60DFFEDEFC22D250E53004B487
:1004D3000801E4F5303099FDC2997599C03099FD52
:1004E300C299F5991204BF221204BF22D250E530FB
:1004F30004B40801E4F5303099FDC2997599C03010
:1005030099FDC299F5991204BF221204BF22D25059
:100513003099FDC2997599C03099FDC299759901B9
:100523007530011204BF221204BF22D2503099FD4C
:10053300C2997599C03099FDC299759900753000BB
:100543001204BF221204BF22D2503099FDC2997502
:1005530099B03099FDC2997599403099FDC299754A
:10056300997F1204BF22D2503099FDC2997599B078
:100573003099FDC2997599403099FDC299759900DA
:100583001204BF22D2503099FDC2997599B03099A7
:10059300FDC2997599403099FDC29975997F1204EE
:1005A300BF22D2503099FDC2997599B03099FDC2DE
:1005B300997599403099FDC2997599001204BF222B
:1005C300D2503099FDC2997599B03099FDC2997591
:1005D30099423099FDC29975997F1204BF22D25076
:1005E3003099FDC2997599B03099FDC299759942B8
:1005F3003099FDC2997599001204BF22D2503099E7
:10060300FDC2997599B03099FDC299759942309997
:10061300FDC29975997F1204BF22D2503099FDC251
:10062300997599B03099FDC2997599423099FDC277
:10063300997599001204BF22D2503099FDC2997561
:1006430099B03099FDC2997599433099FDC2997556
:10065300997F1204BF22D2503099FDC2997599B087
:100663003099FDC2997599433099FDC299759900E6
:100673001204BF22D2503099FDC2997599B03099B6
:10068300FDC2997599433099FDC29975997F1204FA
:10069300BF22D2503099FDC2997599B03099FDC2ED
:1006A300997599433099FDC2997599001204BF2237
:1006B300D2503099FDC2997599B03099FDC29975A0
:1006C30099013099FDC29975997F1204BF22D250C6
:1006D3003099FDC2997599B03099FDC29975990108
:1006E3003099FDC2997599001204BF22D2503099F6
:1006F300FDC2997599B03099FDC2997599013099E8
:10070300FDC29975997F1204BF22D2503099FDC260
:10071300997599B03099FDC2997599013099FDC2C7
:10072300997599001204BF22D2503099FDC2997570
:1007330099B03099FDC2997599023099FDC29975A6
:10074300997F1204BF22D2503099FDC2997599B096
:100753003099FDC2997599023099FDC29975990036
:100763001204BF22D2503099FDC2997599B03099C5
:10077300FDC2997599023099FDC29975997F12044A
:10078300BF22D2503099FDC2997599B03099FDC2FC
:10079300997599023099FDC2997599001204BF2287
:1007A300D2503099FDC2997599D03099FDC299758F
:1007B300997F1204BF22D2503099FDC2997599D006
:1007C3003099FDC2997599001204BF22D250309915
:1007D300FDC2997599D03099FDC29975997F12041C
:1007E300BF22D2503099FDC2997599D03099FDC27C
:1007F300997599001204BF22D2503099FDC29975A0
:1008030099C03099FDC2997599007530001204BFE3
:10081300221204BF22D2503099FDC2997599C0307B
:1008230099FDC2997599007530001204BF22120414
:10083300BF22D2503099FDC2997599C03099FDC23B
:10084300997599017530011204BF221204BF22D297
:10085300503099FDC2997599C03099FDC299759927
:10086300017530011204BF221204BF22D250309905
:10087300FDC2997599C03099FDC299759902753079
:10088300021204BF221204BF22D2503099FDC29932
:100893007599C03099FDC299759902753002120499
:1008A300BF221204BF22D2503099FDC2997599C05C
:1008B3003099FDC2997599037530031204BF221252
:1008C30004BF22D2503099FDC2997599C03099FD69
:1008D300C2997599037530031204BF221204BF2213
:1008E300D2503099FDC2997599C03099FDC299755E
:1008F30099047530041204BF221204BF22D250306F
:1009030099FDC2997599C03099FDC299759904757D
:1009130030041204BF221204BF22D2503099FDC208
:10092300997599C03099FDC299759905753005126D
:1009330004BF221204BF22D2503099FDC299759987
:10094300C03099FDC2997599057530051204BF220F
:100953001204BF22D2503099FDC2997599C03099C3
:10096300FDC2997599067530061204BF221204BFA1
:1009730022D2503099FDC2997599C03099FDC29920
:100983007599067530061204BF221204BF22D25095
:100993003099FDC2997599C03099FDC2997599072F
:1009A3007530071204BF221204BF22D2503099FDC2
:1009B300C2997599C03099FDC29975990775300729
:1009C3001204BF221204BF22D2503099FDC299757E
:1009D30099FA1204BF221204BF22D2503099FDC2E9
:1009E300997599FA1204BF221204BF22D25030998A
:1009F300FDC2997599FB1204BF221204BF22D25083
:100A03003099FDC2997599FB1204BF221204BF22CB
:100A1300D2503099FDC2997599FC1204BF22120479
:100A2300BF22D2503099FDC2997599FC1204BF229E
:100A33001204BF22D2503099FDC2997599C03099E2
:100A4300FDC2990531E531547FF59922D250309991
:100A5300FDC2997599C03099FDC2991531E531549C
:100A63007FF59922D2503099FDC2997599B030998A
:100A7300FDC2997599603099FDC29975990022D28A
:100A8300503099FDC2997599B03099FDC299759905
:100A9300613099FDC29975990022FFE0FFE0FFE004
:100AA300FFE0FFE0FEE1FEE1FEE1FEE1FEE1FDE24B
:100AB300FDE2FDE2FDE2FDE2FCE3FCE3FCE3FCE33B
:100AC300FCE3FBE4FBE4FBE4FBE4FBE4FAE5FAE52B
:100AD300FAE5FAE5FAE5F9E6F9E6F9E6F9E6F9E61B
:100AE300F8E7F8E7F8E7F8E7F8E7F7E8F7E8F7E80B
:100AF300F7E8F7E8F6E9F6E9F6E9F6E9F6E9F5EAFB
:100B0300F5EAF5EAF5EAF5EAF4EBF4EBF4EBF4EBEA
:100B1300F4EBF3ECF3ECF3ECF3ECF3ECF2EDF2EDDA
:100B2300F2EDF2EDF2EDF1EEF1EEF1EEF1EEF1EECA
:100B3300F0EFF0EFF0EFF0EFF0EFF0EFF0EFF0EFBA
:100B4300F0EFF0EFF0EFF0EFF0EFF0EFF0EFF0EFAA
:100B5300F0EFF0EFF0EFF0EFF0EFF0EFF0EFF1EE9A
:100B6300F1EEF2EDF2EDF3ECF3ECF4EBF4EBF5EA8A
:100B7300F5EAF6E9F6E9F7E8F7E8F8E7F8E7F9E67A
:100B8300F9E6FAE5FAE5FBE4FBE4FCE3FCE3FDE26A
:100B9300FDE2FEE1FEE1FFE0FFE0E0FFE3FCE6F95A
:100BA300E9F6ECF3EFF0F2EDF5EAF8E7FBE4FEE14A
:100BB300FFE0FFE0FFE0FFE0FFE0FEE1FEE1FEE13A
:100BC300FEE1FEE1FDE2FDE2FDE2FDE2FDE2FCE32A
:100BD300FCE3FCE3FCE3FCE3FBE4FBE4FBE4FBE41A
:100BE300FBE4FAE5FAE5FAE5FAE5FAE5F9E6F9E60A
:100BF300F9E6F9E6F9E6F8E7F8E7F8E7F8E7F8E7FA
:100C0300F7E8F7E8F7E8F7E8F7E8F6E9F6E9F6E9E9
:100C1300F6E9F6E9F5EAF5EAF5EAF5EAF5EAF4EBD9
:100C2300F4EBF4EBF4EBF4EBF3ECF3ECF3ECF3ECC9
:100C3300F3ECF2EDF2EDF2EDF2EDF2EDF1EEF1EEB9
:100C4300F1EEF1EEF1EEF0EFF0EFF0EFF0EFF0EFA9
:100C5300F0EFF0EFF0EFF0EFF0EFF0EFF0EFF1EE99
:100C6300F1EEF2EDF2EDF3ECF3ECF4EBF4EBF5EA89
:100C7300F5EAF6E9F6E9F7E8F7E8F8E7F8E7F9E679
:100C8300F9E6FAE5FAE5FBE4FBE4FCE3FCE3FDE269
:100C9300FDE2FEE1FEE1FFE0FFE0204D757A796BB6
:100CA300616E7420312076312E3020323030362D73
:100CB30031302D3032202863294164616D20536D1A
:100CC30069616C656B206A616E6B6F6D757A796BA8
:100CD300616E744077702E706C207777772E736D0A
:100CE30069616C656B2E7072762E706C2057737A07
:100CF300656C6B6965207072617761207A617374CA
:100D0300727A657A6F6E652E204A616B69656B6FC7
:100D13006C7769656B207A6173746F736F77616E3B
:100D23006961206B6F6D657263796A6E65206B6FA5
:100D33006475206E6965646F7A776F6C6F6E652E6C
:100D430020416C6C20526967687473205265736527
:100D5300727665642E204672656520666F72206E1A
:100D63006F6E20636F6D6D65726369616C206F6E6A
:040D73006C792E2049
:00000001FF
